:0300000002477E36
:0C477E0078FFE4F6D8FD7581630247C5A2
:101E74000A53746172743A20004950436F6E6E6560
:101E840063745245510A004950436F6E6E65637422
:101E9400003E432C562C43432CC0E4E0EFF2E5F023
:101EA40020D1E8EDEAEEEC49500A003E432C4D41C6
:101EB400432C25303262583A25303262583A253064
:101EC4003262583A25303262583A25303262583AF2
:101ED40025303262582C4D414320E0E4F0E5F10A0C
:101EE400003E432C5645522C20332E3020EEF22057
:101EF40025732025732CC2E5F0F1E8FF204950201A
:101F0400ECEEE4F3EBFF0A004A756E203232203225
:101F14003030370030383A34383A3130003E432CD0
:101F24004C442C50524F473A20202020202020207F
:101F3400202020202020202020202020202020209D
:101F4400202020202020202020202020202020208D
:101F5400202020202020202020202020202020207D
:101F6400202020202020202020202020202CC4E0FD
:101F7400F2E020EFF0EEF8E8E2EAE828F4E0E9EB3A
:101F8400290A003E2A2C312CCEF1EDEEE2EDFBE5E0
:101F940020EFE0F0E0ECE5F2F0FB20F1E5F2E5E221
:101FA400EEE3EE20E8EDF2E5F0F4E5E9F1E00A0015
:101FB4003E412C4130312C2562752E2562752E252B
:101FC40062752E2562752C495020E0E4F0E5F1207D
:101FD400E0E4E0EFF2E5F0E00A003E412C4130326B
:101FE4002C2562752E2562752E2562752E25627547
:101FF4002C495020E0E4F0E5F120EEF1ED2E20F143
:10200400E5F0E2E5F0E00A003E412C4130332C25B6
:1020140062752E2562752E2562752E2562752C49F2
:102024005020E0E4F0E5F120F0E5E72E20F1E5F0C2
:10203400E2E5F0E00A003E412C4130342C25627583
:102044002E2562752E2562752E2562752CCCE0F145
:10205400EAE020F1E5F2E80A003E412C4130352C5B
:102064002562752E2562752E2562752E2562752CC6
:10207400D8EBFEE70A003E532C4130362C2562751E
:102084002CC2F0E5ECFF20EEE6E8E42E20EAE2E8DC
:10209400F2E0EDF6E8E820282A3130ECF1290A00D4
:1020A4003E2A2C312CC4EEEF2E20EFE0F0E0ECE5DC
:1020B400F2F0FB20F1E5F2E5E2EEE3EE20E8EDF2EA
:1020C400E5F0F4E5E9F1E00A003E422C5330312C0E
:1020D4002562752CC6E4E0F2FC20E7E0EFF0EEF1B7
:1020E400E020F1EEE5E4E8EDE5EDE8FF20EEF22096
:1020F400F1E5F0E2E5F0E00A003E422C5330322CE8
:102104002562752C43E2FFE7FC20F120F1E5F0E2C3
:10211400E5F0EEEC20EDE520EFEEE4E4E5F0E6E8B2
:10212400E2E0F2FC0A003E422C5330332C25627567
:102134002CCFE5F0E5E7E0EFF3F1EA20EFF0E8205B
:10214400EFEEF2E5F0E520F1E2FFE7E820F120F11F
:10215400E5F0E2E5F0EEEC0A003E422C5330342C7C
:102164002562752CCDE5F220EFE5F0E5E4E0F7E833
:1021740020E4E8E0E3EDEEF1F2E8EAE820E220F121
:10218400E5F0E2E5F00A003E422C5330352C25629E
:10219400752CCAE0EDE0EB20F8E8F0EEEAEEE2E5BB
:1021A400F8E0F2E5EBFCEDEEE3EE20EEE1ECE5ED3C
:1021B400E00A003E532C5330362C25303262582529
:1021C4003032625825303262582530326258253018
:1021D40032625825303262582C4D414320E0E4F0FD
:1021E400E5F120F8E8F0EEEAEEE2E5F8E0F2E5EBFE
:1021F400FCEDEEE3EE20EEE1ECE5EDE00A003E4519
:102204004E440A0044756D70582020202020303040
:10221400203031203032203033203034203035200B
:1022240030362030372030382030392030412030CB
:10223400422030432030442030452030460A003AC2
:1022440020000A0044756D70442020202020303086
:1022540020303120303220303320303420303520CB
:10226400303620303720303820303920304120308B
:10227400422030432030442030452030460A004577
:102284007272206B657900526420656570726F6D9F
:102294000A005264204D454D0A00526420436F6485
:1022A400650A0044656275674950204F4E0A004430
:1022B400656275674950204F46460A004465627559
:1022C4006755736572204F6E0A00446562756755E1
:1022D400736572204F46460A0044656275674D7304
:1022E40067204F6E0A0044656275674D7367204F1F
:1022F40046460A00436F6E666967206C6F636B2104
:102304000A00577220656570726F6D0A0020536170
:10231400766520656570726F6D210A0045727220C2
:102324004D414321004C6F61643E3E002A003C4114
:1023340030313D003C4130323D003C4130333D00C2
:102344003C4130343D003C4130353D003C41303669
:102354003D004E4F4950004C494E4B434F4E545252
:10236400005452415353004652004E4F4C494E4B79
:1023740000494E49004E4F4449414700003C21006A
:102384003C5330313D003C5330323D003C533033FC
:102394003D003C5330343D003C5330353D003C530C
:1023A40030363D00FF2356FF235BFF2365FF236B7D
:0C23B400FF236EFF2375FF2379FF2380B9
:06516200016000015E0087
:1050F600C2AFC28E758900438910758BFF758DB757
:07510600D2ABD28ED2AF2222
:03001B000246E8B2
:1046E800C0E0C083C082C0D0C2AFC28E758BFF75D8
:1046F8008DB720190675A61E75A6E1055ED215E5CB
:104708006060020560E55FD394014002155F0563B0
:10471800E563540F704AD220E563543F7014D213F6
:10472800906ECCE0600C04F0E0D394B44004C2AFC7
:1047380080FE906EC7E0600204F0906943E060027A
:1047480014F0906ECDE0D394014003E014F03018DB
:10475800020561E562D394644004D21980020562BF
:10476800E55DD394014002155DD28ED2AFD0D0D092
:0647780082D083D0E03284
:10125D00C291C290D2B5C21D7D027C007F07125093
:10126D008A8F27E527646060097D017F6012501E1B
:10127D00D21DE4FDFC7F0B12508A8F27E52730E647
:10128D00097D04E4FF125042D21D7D017C007F07D1
:10129D0012508A8F27E5277008FD7FFF12501ED24E
:1012AD001D301D03126000C2AFC288C2A8C2AA12AF
:1012BD004A13906B80E0B4FA09A3E064CE70030288
:1012CD001354E4F52774782527F582E4346BF58300
:1012DD00E4F00527E527B443EC906B8074FAF0A396
:1012ED0074CEF0A374CCF0906B86740AF0E4A3F086
:1012FD00A304F0A3F0906B8B7403F0A374CCF09067
:10130D006B7C74FFF0A3F0A3F0E4A3F0906B9774E3
:10131D0005F0E4F527E5272401FFE433FE74782575
:10132D0027F582E4346BF583E0FD1250DD0527E5EA
:10133D0027C3944340DFE4F5A775A61E75A6E1907B
:10134D007FF0F0A3F080FED2AF906B8B7403F0A30F
:10135D0074CCF0E4906B8AF01240AAEF6003123265
:10136D002EC2B5123421C219124D7F906B97E0C376
:10137D00940350037403F0D21FD21ED21DD29320BA
:10138D001D077E1E7F74124190E4906DB7F01250D0
:10139D00F6C2AFA37408F0906AF67424F0E4A3F0DB
:1013AD00906B80E0906AF8F0906B81E0906AF9F0B4
:1013BD00906B82E0906AFAF0906B83E0906AFBF09C
:1013CD00906B84E0906AFCF0906B85E0906AFDF084
:1013DD00755F01E4906DB9F0C21AC21BD2AF75A74B
:1013ED000775A61E75A6E1124FF8201D19AF277EB1
:1013FD00007D03124271E4FF12459C7E6B7FB7E4C2
:10140D00FB7D0112434B906ECCE060037401F0E460
:10141D00906943F0A37455F0A37481F0E4F561E491
:10142D00F562906943E0700312271C906ECDE0B415
:10143D0001119080007410F0E4906ECDF0D21DD2A9
:10144D001ED21F908008E0F52730E405D21A7410E3
:10145D00F0E52730E508D21C9080087420F0E527D0
:10146D0030E608D21B9080087440F0E561D39403F8
:10147D004023908002E4F0908001F0908000F0E530
:10148D0061D39406400FE4F561C216906DB9F07505
:10149D005F01124D7F9080A0E07003124B0C908085
:1014AD00B8E070031246469080D0E07003124CB93C
:1014BD00908000E07013301A10123FA6906B73EFFE
:1014CD00F0D394004003120A1A908002E070069047
:1014DD008000E06005D21802142CC218E4F561906A
:1014ED006943E0600302142C301C12123AD5906B44
:1014FD0073EFF0D394004005E0FF125135201B032C
:10150D00021682123960906B73EFF0700302142C87
:10151D00906ECCE060037401F0906BB7E054BF2483
:10152D007F70030215EE1470030215CF24026003C1
:10153D00021621201D077E1E7F7D124190302179DC
:10154D00201676906B8FE07006906B93E0605B9049
:10155D006EC3E0FF906B8FE0B50724906EC4E0FE84
:10156D00906B90E0B50618906EC5E0FE906B91E023
:10157D00B5060C906EC6E0FE906B92E06E602B90FF
:10158D006B93E06F7033906EC4E0FF906B94E0B599
:10159D000727906EC5E0FF906B95E0B5071B906E29
:1015AD00C6E0FF906B96E0B5070F906DB97401F032
:1015BD00120021755F01021682906EC374FFF00256
:1015CD001682906EBBE0FF906BB9E06F6003021660
:1015DD0082906EBBE004F0E4F55F906DB7F00216FB
:1015ED0082301603021682906B86E0700302142C73
:1015FD00125169D216E4F55F906DB7F0906EC70485
:10160D00F0E4906EBAF0A3F0201D6A7E1E7F8B125F
:10161D0041908061301652906BB7E020E74B906B94
:10162D00B9E0FF906EBAE0FE6F600D906EC2E07093
:10163D0007EE146F703F8013906EBAE004F0906B5C
:10164D0073E0FFD394044003124EB790683F748249
:10165D00F0A37401F0906BB9E0906841F07E687F63
:10166D003F7D03124A9102142C3021092016069059
:10167D006EC374FFF0201603021737E55F706B120F
:10168D004EF5EF60207E6C7FB7906CB8E02404FDC2
:10169D00124A91906EC2E0600302142C906B97E099
:1016AD00F55F02142C906EC7E0D3943C403C906ED5
:1016BD00C2E07036906EC704F0906AF5E0702B12A0
:1016CD00514FE4906CB7F0A37412F0906EBBE090A4
:1016DD006CB9F0A374FDF090694663A201906CBBE8
:1016ED0063A2017F121236E5809B125144EF601503
:1016FD0090683F7483F0E4A3F07E687F3F7D021213
:10170D004A9102142CE55F6401600302142C906D64
:10171D00B7E004F0E0C394055003021692C216E43C
:10172D00906DB9F012002102142CE55F6401600385
:10173D0002142C906DB9E014604024FE603C1470CE
:10174D000302181F2404600302142CE4F561202108
:10175D0013906DB97404F0906DB7E05401F0755F9E
:10176D000102142CE4906DB9F0906DB704F0755F23
:10177D00C8906EC374FFF002142C906EC3E070031A
:10178D0002180E906CB77480F0906CB97401F0E48F
:10179D00A3F0A304F0A37430F0A3747BF0E4F52759
:1017AD0074BE2527F582E4346CF583747DF074BF27
:1017BD002527F582E4346CF583E4F0E527240790C2
:1017CD006CB8F07C6E7DC3906B8BE0FAA3E0FB7F71
:1017DD000212488F7E6C7FB7E5272409FD124A91CE
:1017ED00906EC2E0601B125169D216E4F55F906DE8
:1017FD00B7F0906EC704F0E4906EBAF0A3F0021447
:10180D002C906DB97404F0906B97E02432F55F0263
:10181D00142C9080027410F0755F03906DB7E06426
:10182D0001FFF0906DB97401F0EF7019906B93E0BA
:10183D006013FCA3E0FDA3E0FEA3E0FF906EC312D6
:10184D002BC002142C906B8FE0FCA3E0FDA3E0FEF7
:0E185D00A3E0FF906EC3122BC002142C80FE7D
:01186B00225A
:100A1A00906BB8E0B444047F0180027F00906BB70A
:100A2A00E0B447047E0180027E00EE5F604A906B6C
:100A3A0080E0906BB9F0906B81E0906BBAF0906BAC
:100A4A0082E0906BBBF0906B83E0906BBCF0906B94
:100A5A0084E0906BBDF0906B85E0906BBEF0906B7C
:100A6A00B87452F0906AEF63A2019080A863A20161
:100A7A007F061236E5021253906B73E0C394085056
:100A8A000302125C906B80E0FF906BB9E06F600329
:100A9A0002125C906B81E0FF906BBAE06F60030218
:100AAA00125C906B82E0FF906BBBE06F60030212F6
:100ABA005C906B83E0FF906BBCE06F600302125C9A
:100ACA00906B84E0FF906BBDE06F600302125C9054
:100ADA006B85E0FF906BBEE06F600302125C906B67
:100AEA00B8E0B44415906AEFE0B4FF0E63A2019037
:100AFA0080A863A2017F061236E5906ECCE06003FF
:100B0A007401F0906ECD7464F0906BB87452F090EA
:100B1A006BB7E0646D6003020C977BFF7A1E7995D0
:100B2A001224227BFF7A1E79AF906B80E0F530A306
:100B3A00E0F531A3E0F532A3E0F533A3E0F534A301
:100B4A00E0F5351224227530FF75311F75320C75A8
:100B5A0033FF75341F7535187BFF7A1E79E5122429
:100B6A00227BFF7A1F79211224227BFF7A1F798741
:100B7A001224227BFF7A1F79B4906B86E0F530A3AA
:100B8A00E0F531A3E0F532A3E0F5331224227BFF2E
:100B9A007A1F79DE906B8FE0F530A3E0F531A3E0A0
:100BAA00F532A3E0F5331224227BFF7A20790C90E8
:100BBA006B93E0F530A3E0F531A3E0F532A3E0F55D
:100BCA00331224227BFF7A20793A906B7CE0F5304D
:100BDA00A3E0F531A3E0F532A3E0F5331224227B3A
:100BEA00FF7A20795D906B78E0F530A3E0F531A3C8
:100BFA00E0F532A3E0F5331224227BFF7A20797ADA
:100C0A00906B97E0F5301224227BFF7A2079A412A8
:100C1A0024227BFF7A2079CDA221E433F5301224F5
:100C2A00227BFF7A2079FD906EC2E0F530122422F1
:100C3A007BFF7A21792A906ECCE0F5301224227B50
:100C4A00FF7A21795D906AF5E0F5301224227BFF64
:100C5A007A21798BA214E433F5301224227BFF7AAD
:100C6A002179B7906EBCE0F530A3E0F531A3E0F549
:100C7A0032A3E0F533A3E0F534A3E0F535122422DC
:100C8A00123EA17BFF7A22790212242222906BB7AC
:100C9A00E0644C70527E227F08124190906BBFE054
:100CAA00F528A3E0F529E4F52A7D03AF29AE281239
:100CBA0042717E227F43124190AE28AF29E4FB7D28
:100CCA001012434B7E227F4612419074102529F55B
:100CDA0029E43528F528052AE52AC3941040CA7E56
:100CEA00227F4612419022906BB7E0646C705CF5EB
:100CFA002C7E227F48124190E4F52BAF2C7E007D9A
:100D0A00031242717E227F43124190E4F52AA82CF5
:100D1A00E6FF74C1252AF582E4346BF583EFF0050A
:100D2A002C052AE52AB410E67E6B7FC1E4FB7D1010
:100D3A0012434B7E227F46124190052BE52BC3942A
:100D4A000840B87E227F4612419022906BB7E06439
:100D5A004B7061F52A74A9252AF582E4346BF58370
:100D6A00E0603274A9252AF582E4346BF583E0F455
:100D7A00602374A9252AF582E4346BF583E0FF74B5
:100D8A00BF252AF582E4346BF583E0B50710052AFE
:100D9A00E52AB408C09069437432F0021253906B8A
:100DAA00B77421F0301D030212537E227F83124151
:100DBA0090021253906BB7E0B4521A201D077E229C
:100DCA007F8B124190906BB77472F07E6B7FB77D08
:100DDA000812491322906BB7E064497045201D0739
:100DEA007E227F96124190906BBFE0F528A3E0F532
:100DFA0029E4F52A852982852883E0FF74C1252AFA
:100E0A00F582E4346BF583EFF00529E529700205D4
:100E1A0028052AE52AB480DC7E6B7FB77D8A1249D1
:100E2A001322906BB7E064437079A3E06452704672
:100E3A00201D077E227F9E124190906BBFE0F5280D
:100E4A00A3E0F529E4F52A852982852883E493FF1E
:100E5A0074C1252AF582E4346BF583EFF00529E5A0
:100E6A002970020528052AE52AB480DB7E6B7FB744
:100E7A007D8A12491322906BB8E06457600302120C
:100E8A005C906BBFE0F528A3E0F52974C1252AF52B
:100E9A0082E4346BAD82FC7B80AF29AE28124F6BA3
:100EAA00021253906BB7E064446003020F3E906BEA
:100EBA00BFE0FF64447003021253EFB4310CC21D49
:100ECA007E227FA7124190021253906BBFE0B4308A
:100EDA000CD21D7E227FB3124190021253906BBF37
:100EEA00E0B4320CD21E7E227FC01241900212530D
:100EFA00906BBFE0B4330CC21E7E227FCE124190AB
:100F0A00021253906BBFE0B4340CD21F7E227FDDF5
:100F1A00124190021253906BBFE0B4350CC21F7E8F
:100F2A00227FEA124190021253906BBFE0FF120037
:100F3A001E021253906943E07013201D077E227F20
:100F4A00F8124190906BB77421F0021253906943E2
:100F5A007432F0906BB7E0FFB45104C2AF80FEEF79
:100F6A0064577045201D077E237F06124190906BBF
:100F7A00C0E0906B73F0E4F52A906B73E0FFE52A0A
:100F8A00C39F400302125374C1252AF582E4346BCD
:100F9A00F583E0FF906BBFE0252A24EEF582E43466
:100FAA0069F583EFF0052A80D0906BB7E06453604F
:100FBA0003021061201D077E237F11124190906B5E
:100FCA0080E0FF9069F7E06F703C906B81E0FF90E2
:100FDA0069F8E06F7030906B82E0FF9069F9E0B5D4
:100FEA000724906B83E0FF9069FAE0B50718906BCD
:100FFA0084E0FF9069FBE0B5070C906B85E0FF90F9
:10100A0069FCE06F6016906BB77421F0301D030223
:10101A0012537E237F20124190021253E4F52AE4F0
:10102A00F562AF2AFE74EE252AF582E43469F58367
:10103A00E0FD1250DD052AE52AC394FE40E1C2AF65
:10104A00E4907FF0F0A3F0907FFD74AAF0A374FF00
:10105A00F0A37455F080FE906BB7E0644F704C902B
:10106A006BBFE0F528A3E0F529E5294528700A2099
:10107A001D077E237F29124190201D077E237F3082
:10108A00124190E4F52A74C1252AF582E4346BF5FD
:10109A0083E0852982852883F00529E529700205E0
:1010AA0028052AE52AB480DE021253906BB7E0FFC6
:1010BA00B44521906BBFE0FDA3E0907FF0CDF0A393
:1010CA00EDF0C2AF907FFD74AAF0A374FFF0A37491
:1010DA0055F080FEEF64656003021253906BBFE027
:1010EA00FFA3E0907FF0CFF0A3EFF0E4F528F52915
:1010FA00D3907FF1E09529907FF0E095284020E495
:10110A00F5622529FFE5283401FE85298285288391
:10111A00E0FD1250DD0529E5297002052880D17EFF
:10112A00237F3212480AEF4E6020120003906B862A
:10113A00EFF0120003906B87EFF0120003906B88B8
:10114A00EFF0120003906B89EFF07E237F3812488C
:10115A000AEF4E6020120003906B8FEFF01200032B
:10116A00906B90EFF0120003906B91EFF012000376
:10117A00906B92EFF07E237F3E12480AEF4E60207A
:10118A00120003906B93EFF0120003906B94EFF050
:10119A00120003906B95EFF0120003906B96EFF03C
:1011AA007E237F4412480AEF4E6020120003906BA0
:1011BA007CEFF0120003906B7DEFF0120003906B4E
:1011CA007EEFF0120003906B7FEFF07E237F4A12CE
:1011DA00480AEF4E6020120003906B78EFF012007D
:1011EA0003906B79EFF0120003906B7AEFF0120024
:1011FA0003906B7BEFF07E237F5012480AEF4E601C
:10120A0008124DD8906B97EFF0E4F52AE4F562E501
:10121A002A2401FFE433FE7478252AF582E4346B2C
:10122A00F583E0FD1250DD052AE52AC3944340DC2C
:10123A00C2AFE4907FF0F0A3F0907FFD74AAF0A310
:10124A0074FFF0A37455F080FE7E6B7FB77D0812A1
:02125A00491336
:01125C00226F
:104F3300AE07EEC39430400BEED394395005EE2404
:104F4300D0FF22EEC39461400BEED394665005EE7E
:104F530024A9FF22EEC39441400BEED3944650059F
:084F6300EE24C9FF22AF062273
:1050C300906AEEE004F07006906AEDE004F0906AF6
:0A50D300EDE0FEA3E0FF1250A7225B
:100003001250C3124F33EFC454F0FEC0061250C354
:08001300124F33D0E02FFF2251
:104DD8001250C3906946EFF01250C3906947EFF044
:104DE8001250C3906948EFF01250C3906949EFF030
:104DF8001250C390694AEFF01250C390694BEFF01C
:104E08001250C390694CEFF01250C390694DEFF007
:104E1800E4A3F0F533F534F535F5367B017A697995
:054E2800461237BC2218
:04480A008E2D8F2E32
:10480E00906AEDE4F0A374FFF01250C3EF606EF403
:10481E00606B852E82852D83E493B507EC752F0191
:10482E00E52E252FF582E4352DF583E49360259052
:10483E006AEEE0252FFF906AEDE03400FE1250A7DD
:10484E00E52E252FF582E4352DF583E493B5070487
:10485E00052F80CCE52E252FF582E4352DF583E44A
:10486E009370A6E52F24FFFFE434FFFE906AEEE07E
:10487E002FF0906AEDE03EF07E007F0122E4FEFF15
:01488E002207
:1040AA007E237F8112480AEF4E70037F01227E230E
:1040BA007F8412480AEF4E600C1250C3EF24D024BA
:1040CA00FF92218002D2217E237F8A12480AEF4E74
:1040DA00600C1250C3EF24D0906EC2F08005E490B9
:1040EA006EC2F07E237F9012480AEF4E600C125087
:1040FA00C3EF24D0906ECCF08005E4906ECCF07EB5
:10410A00237F9612480AEF4E600C1250C3EF24D058
:10411A00906AF5F08005E4906AF5F07E237F9C12A0
:10412A00480AEF4E600C1250C3EF24D024FF9214B9
:10413A008002C214906B8063A201906EBC63A201DC
:10414A007F061236E530143B7E237FA212480AEF1F
:10415A004E6030120003906EBCEFF0120003906EB6
:10416A00BDEFF0120003906EBEEFF0120003906EE6
:10417A00BFEFF0120003906EC0EFF0120003906ED2
:06418A00C1EFF07F0022EE
:10322E00C214E4906ECCF0D221C217906EC2F09010
:10323E006AF5F0906B8063A201906EBC63A2017F71
:10324E00061236E5E4F528E52875F003A424A8F562
:10325E0082E43423F583E493FB740193FA740293AE
:10326E00F9122A387003023420E4F529F52AFD7488
:10327E006E2DF582E43469F583E0FF700302341B92
:10328E00E52875F003A424A8F582E43423F583E43D
:10329E0093FB740193FA740293F985298275830066
:1032AE00122A51FEEFB50608752A010529023417B8
:1032BE00E52A7003023417EE6003023412E5282467
:1032CE00FE60281470030233FA1470030233FE14E6
:1032DE00700302340614700302340A2405600302DC
:1032EE00341B906ECC7401F002341BD214746E2D0C
:1032FE00F582E43469F583E0FF642D700302341B1C
:10330E00124F33EFC454F0FC746F2DF582E4346920
:10331E00F583E0FF124F33EF2C906EBCF074702DDE
:10332E00F582E43469F583E0FF124F33EFC454F0B5
:10333E00FC74712DF582E43469F583E0FF124F338E
:10334E00EF2C906EBDF074722DF582E43469F58326
:10335E00E0FF124F33EFC454F0FC74732DF582E48A
:10336E003469F583E0FF124F33EF2C906EBEF0748C
:10337E00742DF582E43469F583E0FF124F33EFC408
:10338E0054F0FC74752DF582E43469F583E0FF1278
:10339E004F33EF2C906EBFF074762DF582E43469C6
:1033AE00F583E0FF124F33EFC454F0FC74772DF524
:1033BE0082E43469F583E0FF124F33EF2C906EC038
:1033CE00F074782DF582E43469F583E0FF124F3303
:1033DE00EFC454F0FC74792DF582E43469F583E082
:1033EE00FF124F33EF2C906EC1F08021D217801D4B
:1033FE00906EC27401F08015C2218011906AF5742E
:10340E0001F08009E4F52AF5290D02327D05280226
:02341E00325525
:013420002289
:104E2D00906DB8E0C3947C503D906DB8E0FE04F0F9
:104E3D0074F62EF582E4346AF583EFF0BF0A2790FD
:104E4D006DB8E0FF04F074F62FF582E4346AF58353
:104E5D00E4F0906DB8E0FF124995906DB87408F0CC
:074E6D00906AF7E004F02257
:104D7F009080007480F0906B7863A201F583F582C8
:104D8F0063A2017F081236E5906B8063A2019080C9
:104D9F008863A2017F0A1236E5908092E4F0A37433
:104DAF0032F0A37401F0906B8AE0FF9080B1F09025
:104DBF0080E1EFF09080957455F0A3F0908000742F
:094DCF0001F09080097470F022DB
:104B0C00908009E04410F09080A0E0706C9080A13F
:104B1C007482F09080A874FFF0A3F0A3F0A3F07F50
:104B2C00039080AEEFF07FCBA3EFF07F039080ACCF
:104B3C00EFF0A374CBF09080007402F0906FEC1245
:104B4C002BCC00000000906FECE0908040F0906F58
:104B5C00EDE0908041F0906FEEE0908042F0906F2D
:104B6C00EFE0908043F0A3E4F0A3F0A3F0A3F09067
:094B7C008018F0A3F0A3F0A3F0EF
:014B8500220D
:104CB900908009E04440F09080D17482F0906B8B31
:104CC900E0FF9080DEF0906B8CE0FF9080DFF09049
:104CD90080027402F0906FF0122BCC00000000905B
:104CE9006FF0E0908058F0906FF1E0908059F0906B
:104CF9006FF2E090805AF0906FF3E090805BF0A340
:104D0900E4F0A3F0A3F0A3F0908030F0A3F0A3F0B7
:024D1900A3F005
:014D1B002275
:10464600908009E04420F09080B8E060030246E7DD
:104656009080B97482F07F039080C6EFF07FCDA37F
:10466600EFF07F039080C4EFF0A374CDF030022208
:10467600906B8FE09080C0F0906B90E09080C1F0DE
:10468600906B91E09080C2F0906B92E09080C3F0C6
:10469600800C9080C074FFF0A3F0A3F0A3F090808C
:1046A600017402F0906FF4122BCC00000000906FA2
:1046B600F0E090804CF0906FF1E090804DF0906FBC
:1046C600F2E090804EF0906FF3E090804FF0A3E41C
:1046D600F0A3F0A3F0A3F0908024F0A3F0A3F0A33E
:0146E600F0E3
:0146E70022B0
:10488F008C288D29A907EAFDE975F018A424ACFF3F
:10489F00E5F034808F82F583EDF0EBFDE975F018CC
:1048AF00A4FFAEF024ACFBEE34808B82F583A3ED36
:1048BF00F08529828C83E0FDEF24A8FFEE3480FE83
:1048CF008F82F583EDF08529828C83A3E08F828E12
:1048DF0083A3F0852982852883A3A3E0FDE975F0E2
:1048EF0018A424A8FFE5F03480FE8F82F583A3A3DC
:1048FF00EDF08529828C83A3A3A3E08F828E83A3FF
:04490F00A3A3F0224C
:064913008D2DAB07AA0682
:10491900906FECE0FCA3E0FDA3E0FEA3E0F5318E8F
:10492900308D2F8C2EAE02AF038E838F8263A2014E
:10493900E530540744C0F58385318263A201AF2D68
:1049490012374E908000E020E5F9E4FCFDFEE531E8
:10495900252DF531EE3530F530ED352FF52FEC35C8
:104969002EF52E908040E52EF0A3E52FF0A3E5303B
:10497900F0A3E531F09080007420F0AF31AE30AD96
:0B4989002FAC2E906FEC122BC0AF2D56
:014994002200
:064A91008D28AB07AA0608
:104A9700906FF0E0FCA3E0FDA3E0FEA3E0F52C8E11
:104AA7002B8D2A8C29AE02AF038E838F8263A201DE
:104AB700E52B540744D0F583852C8263A201AF28E8
:104AC70012374EE4FCFDFEE52C2528F52CEE352BA0
:104AD700F52BED352AF52AEC3529F529908058E58F
:104AE70029F0A3E52AF0A3E52BF0A3E52CF09080AD
:104AF700027420F0AF2CAE2BAD2AAC29906FF012C8
:044B07002BC0AF28E8
:014B0B002287
:02459C008F2965
:10459E00908001E030E5037F0022906FF4E0FCA3F1
:1045AE00E0FDA3E0FEA3E0F52D8E2C8D2B8C2A9042
:1045BE006EBC63A201E52C540744C8F583852D8299
:1045CE0063A2017F06123764E52D2406F52DE4352E
:1045DE002CF52CE4352BF52BE4352AF52A906DBA03
:1045EE0063A201E52C540744C8F583852D8263A28E
:1045FE0001AF29123764E4FCFDFEE52D2529F52DCA
:10460E00EE352CF52CED352BF52BEC352AF52A90C5
:10461E00804CE52AF0A3E52BF0A3E52CF0A3E52DC5
:10462E00F09080017420F0AF2DAE2CAD2BAC2A9003
:07463E006FF4122BC0AF293D
:014645002252
:103FA6009081E0E0F528052805280528052805283C
:103FB60005280528052805280528908010E0F52BFA
:103FC600A3E0F52CA3E0F52DA3E0F52E9081E1E02A
:103FD600F528052805280528052805280528052883
:103FE600052805280528908014E0F52FA3E0F53074
:103FF600A3E0F531A3E0F532E531B52D08E532B59C
:104006002E037F0022E4F528E531540744E0F583CA
:1040160085328263A201906BB763A2017F081237D3
:104026007C906BB963A201906AEF63A2017F0612CE
:1040360036E5906BB7E0F529A3E0F52AE4F528907C
:104046006BB7E0702AA3E024F8F528E5315407445D
:10405600E0F58385328274082582F582E43583F59E
:104066008363A201906BB763A201AF2812377CAEBF
:1040760029E4FCFDE532252AF532E5313EF531ED40
:104086003530F530EC352FF52F908014E52FF0A361
:10409600E530F0A3E531F0A3E532F09080007440FE
:0340A600F0AF2850
:0140A90022F4
:103960009081E6E0F5280528052805280528052882
:1039700005280528052805280528908028E0F52B2E
:10398000A3E0F52CA3E0F52DA3E0F52E9081E7E070
:10399000F5280528052805280528052805280528CF
:1039A00005280528052890802CE0F52FA3E0F530A8
:1039B000A3E0F531A3E0F532E4F528E531B52D0AB1
:1039C000E532B52E05C21B023ABAE531540744F080
:1039D000F58385328263A201906BB763A2017F08F1
:1039E00012377C906BB7E0F529A3E0F52AE52A456C
:1039F0002970099080027410F07F0022906EC3E05D
:103A0000FFF4602D906BB9E06F7076906EC4E0FFAC
:103A1000906BBAE06F706A906EC5E0FF906BBBE090
:103A20006F705E906EC6E0FF906BBCE06F602280AE
:103A300050906BB9E0906EC3F0906BBAE0906EC49A
:103A4000F0906BBBE0906EC5F0906BBCE0906EC6E2
:103A5000F0906BB7E0702AA3E024F8F528E5315424
:103A60000744F0F58385328274082582F582E435B7
:103A700083F58363A201906BB763A201AF2812376D
:103A80007CAE29E4FCFDE532252AF532E5313EF530
:103A900031ED3530F530EC352FF52FAF2EAE2DADA5
:103AA0002CAC2BAB32AA31A930A82FD3122BAF40AC
:103AB000099080027410F07F002290802CE52FF096
:103AC000A3E530F0A3E531F0A3E532F09080027475
:043AD00040F0AF28EB
:013AD40022CF
:103AD5009081E3E0F528052805280528052805280F
:103AE5000528052805280528052890801CE0F52BC4
:103AF500A3E0F52CA3E0F52DA3E0F52E9081E4E0FD
:103B0500F528052805280528052805280528052858
:103B1500052805280528908020E0F52FA3E0F5303D
:103B2500A3E0F531A3E0F532E4F528E531B52D0A3A
:103B3500E532B52E05C21C023C20E531540744E8A8
:103B4500F58385328263A20190684363A2017F0EEB
:103B5500123792906843E0F529A3E0F52A90684B67
:103B6500E0FFF46045906EBCE0FEEF6E706EA3E082
:103B7500FF90684CE06F7064906EBEE0FF90684DFA
:103B8500E06F7058906EBFE0FF90684EE06F704C2C
:103B9500906EC0E0FF90684FE06F7040906EC1E09E
:103BA500FF906850E06F60048032D28D906843E0EA
:103BB500702AA3E024F2F528E531540744E8F5839B
:103BC500853282740E2582F582E43583F58363A2FE
:103BD5000190684363A201AF28123792AE29E4FC35
:103BE500FDE532252AF532E5313EF531ED3530F585
:103BF50030EC352FF52FAF2EAE2DAD2CAC2BAB32D7
:103C0500AA31A930A82FD3122BAF5006E52A452992
:103C150070099080017410F07F0022908020E52FBC
:103C2500F0A3E530F0A3E531F0A3E532F090800193
:053C35007440F0AF280F
:013C3A002267
:044190008E2E8F2FB1
:10419400906FECE0FCA3E0FDA3E0FEA3E0F5358E18
:1041A400348D338C32E535FFE5345407FEE42FF5C6
:1041B40031EE34C0F530853182F5837423F0053156
:1041C400E531700205305330C7F582853083740AB7
:1041D400F00531E531700205305330C7906B8063D0
:1041E400A20185308385318263A2017F0612374E96
:1041F40074062531F531E43530F530852E83852F6D
:104204008263A20185308385318263A20112373231
:10421400908000E020E5F9E4FCFDFE906FECE0F80E
:10422400A3E0F9A3E0FAA3E02FFFEE3AFEED39FD97
:10423400EC38FCEF2408FFE43EFEE43DFDE43CFCE6
:10424400906FEC122BC0906FECE0908040F0906F78
:10425400EDE0908041F0906FEEE0908042F0906F3E
:0C426400EFE0908043F09080007420F0A8
:01427000222B
:06434B008E2E8F2F8D3035
:10435100906FECE0FCA3E0FDA3E0FEA3E0F5368E58
:10436100358D348C33E536FFE5355407FEE42FF502
:1043710032EE34C0F531853282F5837423F0053293
:10438100E532700205315331C7F582853183EBF097
:104391000532E532700205315331C7906B8063A25B
:1043A1000185318385328263A2017F0612374E7403
:1043B100062532F532E43531F531852E83852F829C
:1043C10063A20185318385328263A201AF30123746
:1043D1004E908000E020E5F974082530F530FFE4C7
:1043E100FCFDFEE5362FF536EE3535F535ED353488
:1043F100F534EC3533F533908040E533F0A3E53403
:10440100F0A3E535F0A3E536F09080007420F0AF1D
:0D44110036AE35AD34AC33906FEC122BC0DD
:01441E00227B
:024995008F4150
:10499700906FECE0FCA3E0FDA3E0FEA3E0F5458EFD
:1049A700448D438C42E545FFE5445407FEE42FFF61
:1049B700EE34C0906AF663A201F5838F8263A20189
:1049C700AF4112374E908000E020E5F9E4FCFDFE90
:1049D700E5452541F545EE3544F544ED3543F543C9
:1049E700EC3542F542908040E542F0A3E543F0A361
:1049F700E544F0A3E545F09080007420F0AF45AEA4
:0B4A070044AD43AC42906FEC122BC09A
:014A12002281
:064271008E2D8F2EAB051F
:10427700906FECE0FCA3E0FDA3E0FEA3E0F5348E35
:10428700338D328C31E534FFE5335407FEE42FF5E7
:1042970030EE34C0F52F853082F5837423F0053076
:1042A700E5307002052F532FC7F582852F83EBF07A
:1042B7000530E5307002052F906B8063A201852FD2
:1042C7008385308263A2017F0612374E740625303C
:1042D700F530E4352FF52F532FC7E52D853082852F
:1042E7002F83F00530E5307002052F532FC7F58275
:1042F700852F83E52EF00530E5307002052F532F0B
:10430700C7908000E020E5F9E534240AF534E43568
:1043170033F533E43532F532E43531F53190804009
:10432700E531F0A3E532F0A3E533F0A3E534F090EF
:1043370080007420F0AF34AE33AD32AC31906FEC07
:03434700122BC076
:01434A002250
:1050A700E5D220E0FBC2AF438E2075D2028F828EFD
:0B50B70083E0FFE4F5D2538EDFD2AFA0
:0150C20022CB
:1050DD00E5D220E0FBC2AF43D2028F828E83EDF08A
:0950ED0075D25063D250D2AF22FB
:104A1300E4FDED2401FFE433FE1250A774782DF575
:104A230082E4346BF583EFF00DBD3FE6E4FDED2446
:104A33007FFFE433FE1250A7746E2DF582E43469D0
:104A4300F583EFF0746E2DF582E43469F583E0703D
:104A53001B746E2DF582E43469F5837420F0746F52
:104A63002DF582E43469F583E4F080040DBD80BE46
:104A7300E49069EDF0FDEDFF7E001250A774EE2D7A
:0D4A8300F582E43469F583EFF00DBDFEE926
:014A90002203
:024F6B008B2D8C
:104F6D00A2AF9222C2AF85A22E53A2FE8E838F8254
:104F7D0005A28C838D8274091237AAE52D53A2FEEA
:104F8D0043A2201237AC53A2DF852EA2A22292AFEC
:014F9D00FF14
:014F9E0022F0
:10508A00A2AF9222C2AF8C838D82EF1237AA43A2BB
:0C509A00201237AC53A2DFA22292AFFF1D
:0150A60022E7
:02501E008F28D9
:10502000A2AF9222C2AFE4F5838D8274061237AA32
:10503000E52843A2201237AC53A2DFA22292AF7F11
:01504000016E
:01504100224C
:025042008F28B5
:10504400A2AF9222C2AFE4F5838D82740A1237AA0A
:10505400E52843A2201237AC53A2DFA22292AF7FED
:01506400014A
:015065002228
:10360A00A907E7FFA805EF93C3966008403B74FC3F
:10361A002FFF80F00F08EF93C3966008402B74FBCE
:10362A002FFF80E00F08EF93C3966008401B74FADF
:10363A002FFF80D00F08EF93D3966008400B74F9E0
:10364A002FFF80C01F1F1F1F1FEF54FEF80303F731
:10365A00E893FC08E893FD08E893FE08E893FF2244
:10366A0009E993C39D6008402974FB29F980F1098F
:10367A00E993C39E6008401A74FA29F980E209E9BD
:10368A0093D39F6008400B74F929F980D31919194B
:10369A001919E9C313C313FF22740093F8ECC398F2
:1036AA004024701F740193F8EDC398401970147484
:0E36BA000293F8EEC398400E7009740393F863
:1036C800EFC39840037F00227F0122EDF8E6F0085F
:1036D800A3DFFA22EDF8E0F608A3DFFA22E0A363FD
:1036E800A201F0A363A201DFF475A20022E0A363A4
:1036F800A201F0A363A201E0A363A201F0A363A265
:1037080001E463A201F0A363A201DFE175A2002234
:10371800E0A363A2016DFE936CFDEE058393FC1597
:103728008363A201DFEA75A200227F00E493A3630A
:10373800A201F00F600CA3E583C2E3F58363A20145
:1037480080EA75A20022E0A363A201F0A3E583C288
:10375800E3F58363A201DFEE75A20022E0A363A272
:1037680001F0A3E583C2E4D2E3F58363A201DFECB1
:1037780075A20022E583C2E3F583E0A363A201F00A
:10378800A363A201DFEE75A20022E583C2E4D2E3BF
:10379800F583E0A363A201F0A363A201DFEC75A2A5
:1037A8000022F922C002C004C00612FFF0D006D0E1
:0437B80004D0022215
:104B86000A536572763A00205544502054696D6583
:104B96004750530A00200A444154414752414D3A76
:104BA60020002043414E2054696D654750530A004A
:104BB60020547261737353656E644552520A002025
:104BC6005265496E69742043414E0A002043414EA6
:104BD600283029203E20544F210A002054552030E9
:094BE6000A0020545520310A0098
:03001E00E4FF22DA
:104FD200C28DC2AF438901C28C906EE2E0FF7007BE
:104FE200F58A758CEE800AEFB40A06E4F58A758CB0
:064FF20070D28CD2AF2248
:104F9F00C28DC2AF438901C28C906EE2E0FF7014E4
:104FAF00302F09F58A758CDCC22F8012758A6675D1
:104FBF008CFC800AEFB40A06E4F58A758CDCD28C7F
:034FCF00D2AF223C
:104FF800C230906EE2E0C394645006124C54124FD3
:10500800D212516FD22EE4F558906FEAF0F546F5BA
:065018005CC22FF55A22D4
:104EB700EF24FCF528201D127E4B7F861241907E41
:104EC7006B7FBBE4FBAD2812434B906BBAE0B41F7A
:104ED70003D23022906BBB63A201906F6A63A20179
:0D4EE700AF281236E5852846E4F557C22CA9
:014EF400229B
:0F513500D3EF6480948E5006E55C70028F5C228D
:10271C00208D0302281FC28C202E0302291FE55C8A
:10272C0060519068437D48FF1236DCE548640170C7
:10273C001E90684BE0B4FF0ED231201D127E4B7FF1
:10274C008D1241908009303106E4F55C02291F128C
:10275C004FD2124BEF201D077E4B7F9B12419020D6
:10276C001D0B7E687F43E4FBAD5C12434BE4F55CD0
:10277C0002291FE546605C746E2557F582E4346FC0
:10278C00F583E02405F528D3940E4008E4F546D2F1
:10279C002C02291F746A2557F582E4346FF5837D6A
:1027AC0048AF281236DCE5282557F557E54830E7C1
:1027BC0002D22FE548B40103203106124FD2124B3E
:1027CC00EFE557C39546500302291FE4F546D22C7A
:1027DC0002291FE5596023906ECE7D48FF1236DC2E
:1027EC00E548B40109303106E4F55902291F124FAE
:1027FC00D2124BEFE4F55902291FE55BC3946440F8
:10280C000320160C906EE2E0C394645003124D1C2E
:10281C00124FD2123D6F8F28EF700302291F124FF7
:10282C009FE4F55AE548B4010CD231201D077E4BCC
:10283C007FA8124190E55BC3946E40030228F320FD
:10284C0016030228F3303075E5486442706FE54C8E
:10285C007032E54AC454F0FFE54BC4540F2FF548D1
:10286C00E54BC454F0F549754A0874E3255BF582D1
:10287C00E4346EF5837403255BF55B7D487F0312AE
:10288C0036D3806374E3255BF582E4346EF583E51F
:10289C0028255BF55B7D48AF281236D3301F48C323
:1028AC00E55B9528FFE49400FE74E32FF582746ECB
:1028BC003EAF82FEE4FBAD2812434B802AE548B4C0
:1028CC00420DE54BB40208906AF5E064016018749F
:1028DC00E3255BF582E4346EF583E528255BF55B37
:1028EC007D48AF281236D3301424E54830E7033046
:1028FC00021C906DBA7D48AF281236D3AF28124512
:10290C009CEF700A201D077E4B7FB6124190AF28BA
:10291C00122CFE30201A301315906EE2E0C3946432
:10292C00500C055AE55A94F04004C2AF80FEC22008
:10293C00201503022A34E5586031D3940140041564
:10294C00588028906FEAE004F0E0D39403400D2007
:10295C001D077E4B7FC5124190124FF8201D077E3C
:10296C004B7FD2124190E4F558D22E302D43E559CD
:10297C00703F906ECE04F0A37408F0A37480F0A3A3
:10298C007401F0A37406F0906F65E0906ED3F09034
:10299C006F66E0906ED4F0906F67E0906ED5F0901B
:1029AC006F68E0906ED6F0E4A3F0A3F075590BC2FB
:1029BC002D302B72906F63E07035E5597031906E4D
:1029CC00CE7442F0A37408F0906F64E0906ED0F077
:1029DC00906F69E0906ED1F0A37401F075590620E8
:1029EC001D077E4B7FE1124190906F63E004F090E5
:1029FC006F63E06402702FE559702B906ECE7402F9
:102A0C00F0A37408F0906F64E0906ED0F0A3F0A384
:102A1C007401F0755906201D077E4B7FE81241901A
:0B2A2C00906F63E004F0C2151200265A
:012A3700227C
:104EF500E55B6037E4906CB7F0A3E55BF0906EBBC3
:104F0500E0906CB9F0303006A3741FF08006906C09
:104F1500BA7419F0906EE363A201906CBB63A201B1
:0E4F2500AF5B1236E5E4F55B7F01227F0022D0
:0B514400302C05C22C7F01227F0022CE
:0100210022BC
:06516900E4F55BF54622AF
:0A514F00E4906946F0A3F0A3F022FB
:105066002043616E457247495400200A002043617F
:105076006E457272434821000A000A205265714546
:045086007272210021
:103D6F00E59B541F6020201D1A7E507F66124190E4
:103D7F00E59B541FFF7E007D031242717E507F70C2
:103D8F00124190E4F59BE5BA30E010E4F5B375B15C
:103D9F0080F5B2D22EF558906FEAF0E5CFF47003AC
:103DAF00023E9E752A01E4F529E5CFF4552A7003EA
:103DBF00023E8CE529C454F0F5B1E5B2547F64207E
:103DCF006003023E5DE5B3540FF54C85BC482002FD
:103DDF0016E5BD541FFF131313541FFFE5BD54E029
:103DEF0044184FF5498006E5BD54E0F549E5BDC4DB
:103DFF003354E0FFE5BE131313541F4FF54AE5BECE
:103E0F00C43354E0FFE5BF131313541F4FF54B8515
:103E1F00A34D85A34E85A34F85A35085A35185A39D
:103E2F005285A35385A354E4F5B230020C85AE55E9
:103E3F0085AF5675B3D07F0F22E548547EB5480540
:103E4F0075B350800375B3D0E54C2405FF22E5B25E
:103E5F00549F6023201D207E507F73124190AFB27C
:103E6F007E007D03124271AFB37E007D031242715B
:103E7F007E507F7E124190E4F5B275B3D0E52A25CE
:103E8F00E0F52A0529E529C394085003023DB87FC0
:013E9F000022
:013EA00022FF
:104BEF00200261906EE2E0C39464505675B180E488
:104BFF00F5B3F5B28548BCE54AC4135407FFE54940
:104C0F0054E04FF5BDE54A33333354F8FFE54BC459
:104C1F001354074FF5BEE54B33333354F8F5BF85C7
:104C2F004DA3854EA3854FA38550A38551A38552D0
:104C3F00A38553A38554A3E54C540F2450F5B375A6
:054C4F00580AC22E22EC
:104D1C0020025F75B190E5B220E613201D107E5085
:104D2C007F80124190AFB27E007D03124271E4F598
:104D3C00B3F5B274892515F582E43461F583E0F599
:104D4C00BCE4F5BD748A2515F582E43461F583E085
:104D5C00FF33333354F8F5BE75BF7805150515745C
:104D6C00892515F582E43461F583E07002F515753B
:034D7C00B350220F
:09515900EF6003C29622D29622F7
:104C540043AB01C2E8C2EAE4FFEFC454F0F5B1C3C8
:104C6400EF64809488500575B3D08003E4F5B3E411
:104C7400F5B2F5BCF5BDF5BEF5BFF5C4F5C5F5C691
:104C8400F5C7F5A3F5A3F5A3F5A3F5A3F5A3F5A33C
:104C9400F5A30FBF0EC3906EE2E0FF25E0F5B475F7
:104CA400B50C75B66C75A11275AB0275C13E75C3B2
:044CB400FF75C203C3
:014CB80022D9
:10186C005452414E5A004D41584200525453004478
:10187C00454C4159004D4F4445004B5000545500C8
:10188C0043414E004B5654004154004449520043CE
:10189C00414E4D4F4E00475254494D45005449540A
:1018AC0053005453494E5600003E2A2C312CCFE0A5
:1018BC00F0E0ECE5F2F0FB20F3EFF0E0E2EBFFFE02
:1018CC00F9E5E3EE20EAEEEDF2F0EEEBEBE5F0E01D
:1018DC0020CACF20C8F1E5F2FC0A003E4C2C6B303C
:1018EC00312C25732C43EAEEF0EEF1F2FC20EDE006
:1018FC0020F8E8EDE52043414E2C30202D203530EA
:10190C0030EAE1283530EC292C31202D203530EA15
:10191C00E128353030EC290A0030202D20353030CC
:10192C00EAE1283530EC290031202D203530EAE170
:10193C0028353030EC29003E532C6B30322C25628C
:10194C00752CCCE0EAF12E20E0E4F0E5F120E1EB9F
:10195C00EEEAE020D2D128302D38290A003E532C53
:10196C006B30332C2562752CCCE0EAF12E20E0E4B0
:10197C00F0E5F120E1EBEEEAE020D2C8D228302DE0
:10198C0038290A003E532C6B30342C2562752CCC34
:10199C00E0EAF12E20E0E4F0E5F120E1EBEEEAE004
:1019AC0020D2D328302D38290A003E2A2C312CCFB6
:1019BC00E0F0E0ECE5F2F0FB20EFF0EEF2EEEAEE18
:1019CC00EBE020C3F0E0EDE8F220EFEE20EFEEF0DC
:1019DC00F2F32052533233320A003E4C2C6B30352A
:1019EC002C256C752CD1EAEEF0EEF1F2FC20EEE138
:1019FC00ECE5EDE020EDE020EFEEF0F2F32C3130F1
:101A0C00302C3230302C3330302C3630302C3132CC
:101A1C0030302C323430302C343830302C393630A5
:101A2C00302C31393230302C33383430302C35378F
:101A3C003630302C3131353230300A003E532C6B7D
:101A4C0030362C2562752CCDEEECE5F020CACF207B
:101A5C000A003E422C6730312C2562752CCCE0E319
:101A6C00E8F1F2F0E0EBFC0A003E422C6730322C3D
:101A7C002562752CC8EDE2E5F0F2E8F0EEE2E0F25A
:101A8C00FC20E7EDE0F7E5EDE8FF20D2D10A003EBF
:101A9C00422C6730332C2562752CC8F1EFEEEBFC31
:101AAC00E7EEE2E0F2FC20F0E0F1F8E8F0E5EDED35
:101ABC00FBE920EFF0EEF2EEEAEEEB20F1EE20E2A5
:101ACC00F0E5ECE5EDE5EC0A003E422C6730342CF9
:101ADC002562752CC2FBF1F2E0E2EBFFF2FC205226
:101AEC00545320EFF0E820EFE5F0E5E4E0F7E50AE9
:101AFC00003E532C6730352C2562752CC7E0E4E58D
:101B0C00F0E6EAE020EFE5F0E5E4E0F7E820EFEEC0
:101B1C00F1EBE52052545320282A3130ECF1290AFC
:101B2C00003E532C6730362C2562752C4BEEECECBA
:101B3C00F3F2E8F0F3E5ECE0FF20EBE8EDE8E82069
:101B4C00F1E2FFE7E8202830290A003C21003C6B39
:101B5C0030313D003C6B30323D003C6B30333D004E
:101B6C003C6B30343D003C6B30353D003C6B3036CB
:101B7C003D003C6730313D003C6730323D003C67F6
:101B8C0030333D003C6730343D003C6730353D0020
:101B9C003C6730363D000A41734F55543A2000548F
:101BAC00530A005455204F4B0A0054552044696188
:101BBC00670A005455205265710A00205455205470
:101BCC00696D654F5554210A004154636F6E6E6503
:101BDC0063740A000A4173494E3A20000A43524387
:101BEC00204552523A20000A4E6B703A20000ACF20
:101BFC00F0E8EDFFF2E020EAEEECE0EDE4E020D2DC
:101C0C00D320002020D2D320E7E0EDFFF2EE210A12
:101C1C00000ACDE520EFEEEDFFEB20F2E8EF20EF30
:101C2C00E0EAE5F2E0210A00001123324657657420
:101C3C008C9DAFBECADBE9F81001332256477564A0
:101C4C009C8DBFAEDACBF9E8213002136776445590
:101C5C00ADBC8E9FEBFAC8D9312012037766544580
:101C6C00BDAC9E8FFBEAD8C9425361700415273670
:101C7C00CEDFEDFC8899ABBA524371601405372660
:101C8C00DECFFDEC9889BBAA637240512534061750
:101C9C00EFFECCDDA9B88A9B736250413524160740
:101CAC00FFEEDCCDB9A89A8B8495A7B6C2D3E1F030
:101CBC0008192B3A4E5F6D7C9485B7A6D2C3F1E020
:101CCC0018093B2A5E4F7D6CA5B48697E3F2C0D110
:101CDC0029380A1B6F7E4C5DB5A49687F3E2D0C100
:101CEC0039281A0B7F6E5C4DC6D7E5F48091A3B2F0
:101CFC004A5B69780C1D2F3ED6C7F5E49081B3A2E0
:101D0C005A4B79681C0D3F2EE7F6C4D5A1B08293CF
:101D1C006B7A48592D3C0E1FF7E6D4C5B1A09283BF
:101D2C007B6A58493D2C1E0F0089129B24AD36BF8F
:101D3C0048C15AD36CE57EF78108931AA52CB73E9F
:101D4C00C940DB52ED64FF76028B109926AF34BD8F
:101D5C004AC358D16EE77CF5830A9118A72EB53C7F
:101D6C00CB42D950EF66FD74048D169F20A932BB6F
:101D7C004CC55ED768E17AF3850C971EA128B33A5F
:101D8C00CD44DF56E960FB72068F149D22AB30B94F
:101D9C004EC75CD56AE378F1870E951CA32AB1383F
:101DAC00CF46DD54EB62F97008811A932CA53EB72F
:101DBC0040C952DB64ED76FF89009B12AD24BF361F
:101DCC00C148D35AE56CF77E0A8318912EA73CB50F
:101DDC0042CB50D966EF74FD8B029910AF26BD34FF
:101DEC00C34AD158E76EF57C0C851E9728A13AB3EF
:101DFC0044CD56DF60E972FB8D049F16A920BB32DF
:101E0C00C54CD75EE168F37A0E871C952AA338B1CE
:101E1C0046CF54DD62EB70F98F069D14AB22B930BE
:101E2C00C74ED55CE36AF1780008040C020A060E72
:101E3C000109050D030B070FFF186CFF1872FF1833
:101E4C0077FF187BFF1881FF1886FF1889FF188C05
:101E5C00FF1890FF1894FF1897FF189BFF18A2FF0C
:081E6C0018A9FF18AEFF18B41D
:10510D00EF540F901E3493FEC454F0FEEFC4540FB1
:04511D00932EFF22AC
:0300230002441F75
:0B441F00C0E0C083C082C0D075D01880
:10442A00309852C298756001AF9920074820030B53
:10443A00EF64027040D203D291803A300C04C20C6D
:10444A008024BF0904D20C802CBF0205530C808043
:10445A0024BF0312906616E50CF0630C80530C809F
:10446A00C203C291800F7439250CF582E43466F5D3
:10447A0083EFF0050C30995F30045A906187E0FFB2
:10448A00E50DC39F4008C204D211C2908047D29062
:10449A00AF0D050D74392FF582E43467F583E0F525
:1044AA0010300B1953107F30012830D00830062203
:1044BA00631080801D20061A631080801530011257
:1044CA00E50B5210300606A2D0929B8005A2D0B30B
:0744DA00929B851099C29925
:0944E100D0D0D082D083D0E032AB
:103EA1007BFF7A1879B5122422906EE2E0701475C6
:103EB10030FF7531197532257BFF7A1879E71224A5
:103EC1002280127530FF7531197532347BFF7A18F3
:103ED10079E71224227BFF7A197943906188E0F512
:103EE100301224227BFF7A197969906101E0F53063
:103EF1001224227BFF7A197990906100E0F530124B
:103F010024227BFF7A1979B612242290683DE0FEC3
:103F1100A3E0FFC3E49FFFE49EFEAB07FA3395E005
:103F2100F9F87F007E8C7D0A7C00122B0F8F338E77
:103F3100328D318C307BFF7A1979E61224227BFF96
:103F41007A1A7948906405E0F5301224227BFF7AD1
:103F51001A795E90683BE0F5301224227BFF7A1AD1
:103F61007975A20AE433F5301224227BFF7A1A799B
:103F71009BA205E433F5301224227BFF7A1A79D50E
:103F8100A20FE433F5301224227BFF7A1A79FD85E2
:103F910009301224227BFF7A1B792D90683AE0F5D3
:053FA100301224222271
:103C3B007E1B7F5712480AEF4E70037F0122E490E0
:103C4B006EE2F07E1B7F5A12480AEF4E601512503F
:103C5B00C3BF3106906EE2740AF0BF3206906EE27B
:103C6B007464F07E1B7F6012480AEF4E6008124DA1
:103C7B00D8906188EFF07E1B7F6612480AEF4E608A
:103C8B0008124DD8906101EFF07E1B7F6C12480A31
:103C9B00EF4E6008124DD8906100EFF07E1B7F72E3
:103CAB0012480AEF4E6023124DD8A804A905AA06A4
:103CBB00AB077F007E8C7D0A7C00122B0F122BA191
:103CCB0090683DEEF0A3EFF0800A90683D74FFF032
:103CDB00A374DCF07E1B7F7812480AEF4E6008124B
:103CEB004DD8906405EFF07E1B7F7E12480AEF4E95
:103CFB00600A1250C3EF24D190683BF07E1B7F8487
:103D0B0012480AEF4E600A1250C3EF24D024FF92E0
:103D1B000A7E1B7F8A12480AEF4E600A1250C3EFCD
:103D2B0024D024FF92057E1B7F9012480AEF4E6031
:103D3B000A1250C3EF24D024FF920F7E1B7F9612E2
:103D4B00480AEF4E6005124DD88F097E1B7F9C12DF
:103D5B00480AEF4E600B124DD8906839EEF0A3EF86
:033D6B00F07F00E6
:013D6E002232
:102FA300E4F528E52875F003A42444F582E4341EEF
:102FB300F583E493FB740193FA740293F9122A38AC
:102FC300700302322DE4F52AF52BF529746E2529B9
:102FD300F582E43469F583E0FF7003023228E528C3
:102FE30075F003A42444F582E4341EF583E493FBD3
:102FF300740193FA740293F9852A82758300122A65
:1030030051FEEFB50608752B01052A023223E52B85
:103013007003023223EE600302321EE528B40F0070
:10302300400302322890302FF828287302305C02C4
:1030330030A30230DC0230E102310C02316E023285
:103043002802314002322802319C0231E502321259
:1030530002321602322802321A746E2529F9E43438
:1030630069FA7B01C0031B8B33753400753500E4AB
:10307300F536D0031237BC8F2F8E2E8D2D8C2CABB3
:103083002FAA2EA92DA82C7F007E8C7D0A7C0012EE
:103093002B0F122BA190683DEEF0A3EFF002322824
:1030A300746E2529F582E43469F583E024D09061B8
:1030B30088F0746F2529F582E43469F583E024D020
:1030C300906101F074702529F582E43469F583E099
:1030D30024D0906100F0023228D20F023228746E9D
:1030E3002529F9E43469FA7B01C0031B8B3375345A
:1030F30000753500E4F536D0031237BC8F2F8E2EC2
:103103008D2D8C2C8F09023228746E2529F582E4CB
:103113003469F583E0B43702D20B746F2529F58245
:10312300E43469F583E0FFB44E04C2018002D201A6
:10313300EF64456003023228D206023228746E25FA
:1031430029F9E43469FA7B01C0031B8B337534001E
:10315300753500E4F536D0031237BC8F2F8E2E8DD4
:103163002D8C2C906EE2EFF0023228746E2529F933
:10317300E43469FA7B01C0031B8B33753400753566
:1031830000E4F536D0031237BC8F2F8E2E8D2D8C95
:103193002C906405EFF0023228746E2529F9E4348B
:1031A30069FA7B01C0031B8B33753400753500E46A
:1031B300F536D0031237BC8F2F8E2E8D2D8C2CE439
:1031C300FFFEFDFCAB2FAA2EA92DA82CD3122BAFEB
:1031D300400A906839E52EF0A3E52FF0D20EC20D18
:1031E3008043746E2529F9E43469FA7B01C0031B1B
:1031F3008B33753400753500E4F536D0031237BCD4
:103203008F2F8E2E8D2D8C2C90683BEFF08016D255
:10321300028012D205800EC20A800AE4F52BF52A39
:0A3223000529022FCF0528022FA66F
:01322D00227E
:10342100C22BC210C209C208906184740AF0E490F0
:10343100683CF090683AE024F9FE906839E034FF86
:10344100906303F0A3CEF0E4906186F0C21290661F
:10345100187405F0C22DE4F508906944E0645570D4
:1034610004A3E06481603BE4FF7F409061B9E4F034
:10347100A3DFFCE4FF7F20906619E4F0A3DFFCE406
:10348100FF74062FF582E43466F583E4F0740E2FA1
:10349100F582E43466F583E4F00FBF08E4E4F50E49
:1034A100F50FE4F514F513906302F0906301F0C297
:1034B10004C211C207C203C20CF50D906187F0F579
:1034C10009F50CF560C200C20BC20F90683D74FF94
:1034D100F0A374F4F0750BFFC20EE4906405F09054
:1034E100683BF0D20DC202C205906839F0A374782E
:1034F100F0D20AE4906EE2F0123C3BEF6003122F2F
:10350100A3E4F5157E617F89906188E0F515E515E5
:10351100C394014007E515D394084003E4F515E58C
:103521001560220FEFAC0670010E14F5828C8374C6
:10353100C4F015150FEFAC0670010E14F5828C83E3
:10354100E515F080DA906101E0F515E515C3940108
:103551004007E515D394084003E4F515E51560220D
:103561000FEFAC0670010E14F5828C8374C8F01550
:10357100150FEFAC0670010E14F5828C83E515F082
:1035810080DA906100E0F515E515C394014007E587
:1035910015D394084003E4F515E51560220FEFAC4F
:1035A1000670010E14F5828C8374C2F015150FEFAD
:1035B100AC0670010E14F5828C83E515F080DA0FEC
:1035C100EFAC0670010E14F5828C83E4F08F828ECD
:1035D10083F0F515C2ADF5C9D2CDD2CCC2C9C2CAEC
:1035E100F5CDF5CC90683DE0F5CBA3E0F5CA85CBF0
:1035F100CD85CACCD29ED29CD2CAC2ACC298C29945
:0836010075B81075B710D2ACCA
:01360900229E
:10512100E5126FFF901D34936511F512EF901C3459
:0351310093F511E2
:015134002258
:0244EA008F2E13
:1044EC00E4FC752F61753002F512F511FDEDC395E5
:1044FC002E50170530E530AE2F7002052F14F582C3
:10450C008E83E0FF1251210D80E30530E530AE2F94
:10451C007002052F14F5828E83E512F085308285AA
:10452C002F83E511F0052E052E7E677F39752F61DF
:10453C007530028F828E837402F00FBF00010E0C57
:10454C00E4FDEDC3952E5038853082852F83E0F93C
:10455C0064026008E964036003B9090D8F828E83DD
:10456C007409F00FBF00010E0C8F828E83E9F00FDF
:10457C00BF00010E0C0530E5307002052F0D80C216
:0F458C008F828E837403F00FBF00010E0CAF04FB
:01459B0022FD
:03516F00C2072252
:104E74008F2D20043D300D3AAF2D1244EA90618706
:104E8400EFF0201D127E1B7FA21241907E617F02F3
:104E9400E4FBAD2D12434B300F057F01125159E550
:104EA400096003F55D22E4F50DD204C2992099FD51
:034EB400D299226E
:022CFE008F291C
:102D0000906405E07003022FA2E54824BE70030220
:102D10002F4B24FA7003022ECF24046003022FA24B
:102D2000E54930E703022DBAE54B6068E54AC394F4
:102D3000024003022FA2E54A7007E54B14F52A80F2
:102D400006E54B241FF52AE52A75F004A42405F5B1
:102D500082746335F0F5837D4D7F041236D3E52A06
:102D600075F004A42401F582746235F0F5837D5179
:102D70007F041236D374F9254AF582E43461F58371
:102D80007481F074B9252AF582E43461F583740105
:102D9000F0D208227406254AF582E43466F583747D
:102DA00080F0E54A75F004A42419F582746635F0C4
:102DB000F5837D4D7F041236D322E54C6408600311
:102DC000022FA2E54AC394044003022FA2201D074C
:102DD0007E1B7FAB124190752901E54B5407FFE53F
:102DE00029A807088002C333D8FCF5297408250FE9
:102DF000F50FB50E067408250EF50EE54B547FFF52
:102E0000E54AC43354E02FFE7400250FF582E43404
:102E100060F583EEF0E54BC394805022EF1313135B
:102E2000541FFFE54A25E025E02F2419F582E434FC
:102E300066F583E0FFE529F4FEEF5EF0802EE54BBA
:102E4000547FFF131313541FFFE54A25E025E02F9D
:102E50002419F582E43466F583E04529F0740025F1
:102E60000FF582E43460F583E04480F07401250FAF
:102E7000F582E43460F5837D4D7F041236D3E5524C
:102E8000FEE551FF7C007D0A122A7EEF7405250FB6
:102E9000F582E43460F583EFF07406250FF582E4E3
:102EA0003460F583E553F07407250FF582E4346050
:102EB000F583E554F0301D03022FA27400250FF5B1
:102EC00082E43460AF82FEE4FB7D0812434B22E5CE
:102ED0004B54E064407003022FA2E54A701DE54B9D
:102EE0001313543FFF7401A807088002C333D8FCB2
:102EF0004213906301E04513F08024E54A640160C9
:102F000003022FA2E54B1313543FFF7401A80708D7
:102F10008002C333D8FC4214906302E04514F0E50C
:102F20004A75F020A4FFE54B547F7C002FFFEC3561
:102F3000F0FEEF25E0FFEE33FE74062FF582746499
:102F40003EF5837D4DAF4C1236D322E54BB40113D1
:102F5000201D077E1B7FAF124190E54E04906FEB62
:102F6000F0C22BE54BB40216240EF582E43466F56C
:102F700083E54EF0201D077E1B7FB6124190E54B86
:102F8000B4031F240EF582E43466F583E54EF02089
:102F90001D077E1B7FBF124190302B06906F63741C
:022FA00002F03D
:012FA200220C
:10002600906405E07003020A19301361050A9066B0
:1000360018E0600214F090683CE0600214F09068EA
:100046003BE06008906184E0600214F0C213300E59
:1000560021906839E0FEA3E0FFD3906304E09F900F
:100066006303E09E500CA3E004F07006906303E087
:1000760004F0302B18906185E004F0E0D3940A4038
:100086000C201D077E1B7FC7124190C22BE55DB475
:10009600010EE4F55DF50DD204C2992099FDD299C1
:1000A60030040DE50AD394064009C204D211800338
:1000B600E4F50A200E0302019190683AE024FBFF62
:1000C600906839E034FFFEC3906304E09F906303B9
:1000D600E09E4012906186E0700CC20DFF125159ED
:1000E6009061867401F090683AE024FDFF906839CB
:1000F600E034FFFEC3906304E09F906303E09E40FC
:1001060012906186E0B4010B7F011251599061860D
:100116007402F090683AE024FEFF906839E034FFFC
:10012600FEC3906304E09F906303E09E405D20045D
:100136005A9067397441F0A37454F0A37424F0A361
:100146007443F0A3744FF0A314F0A3F0A37445F026
:10015600A37443F0A37454F0A3740DF0A3740AF0CF
:10016600906187740CF0E4F50DD204C2992099FDD4
:10017600D299E4906303F0A3F0906186F0301D03FA
:10018600020A197E1B7FD51241902230110AC21134
:10019600300F05E4FF125159300403020678E55D7D
:1001A6006003020678200D03020678906184E06001
:1001B6000302067890683BE06007E4906184F08073
:1001C60006906184740AF0301229C212E49061022A
:1001D600F0A37408F0906405E0906104F09066174F
:1001E600E0906105F0A374FEF0A3748FF07F061211
:1001F6004E7422906FEBE0FF6025E4906102F0A35D
:100206007408F0906405E0906104F0A37483F0A391
:10021600EFF0E4A3F0906FEBF07F06124E7422E548
:100226000F650E700302032690683CE0600302042B
:1002360012E50E2408F529E4906102F0A37408F093
:10024600906405E0906104F0A374F0F0A37406F0E6
:10025600A37491F074062529F582E43460F583E0F1
:10026600906108F074072529F582E43460F583E08F
:10027600906109F074012529F582E43460F583E084
:1002860090610AF074022529F582E43460F583E072
:1002960090610BF074032529F582E43460F583E060
:1002A60090610CF074042529F582E43460F583E04E
:1002B60090610DF074002529F582E43460F583E041
:1002C600FF547FFEC39440500BEFC454F00490617A
:1002D6000EF0801674002529F582E43460F583E07B
:1002E600FFC454F0240590610EF074002529F582B0
:1002F600E43460F583E0FFEEC4540F90610FF0EF35
:100306005480FF74052529F582E43460F583E02FD7
:10031600906110F090683C7414F07F0F124E7422B6
:10032600300973906606E0D39400406AE490610257
:10033600F0A37408F0906405E0906104F0A37441A2
:10034600F0A37420F0752B61752C07E4F529741958
:100356002529F582E43466F583E0F52A300A06FF9E
:1003660012510D8F2A852C82852B83E52AF0F4FF06
:10037600E5822408F582E43583F583EFF0052CE564
:100386002C7002052B0529E529C3940840C07F156A
:10039600124E74C20922301073906608E0D394009E
:1003A600406AE4906102F0A37408F0906405E0905E
:1003B6006104F0A37445F0A37420F0752B61752CCD
:1003C6000775290874192529F582E43466F583E052
:1003D600F52A300A06FF12510D8F2A852C82852BAD
:1003E60083E52AF0F4FFE5822408F582E43583F5F7
:1003F60083EFF0052CE52C7002052B0529E529C3B2
:10040600941040C07F15124E74C2102220080302B9
:1004160005159061FAE0FF9061F9E04F5401D3941D
:10042600005003020515E4F52974B92529F582E47F
:100436003461F583E0700302050774B92529F58256
:10044600E43461F583E4F0906102F0A37408F0905F
:100456006405E0906104F0A374F0F0A37403F0A3C4
:100466007491F0E529C4540F2408A3F0E529540F2C
:10047600A3F0E52925E025E0F5292401F582E434F9
:1004860062F583E090610AF074022529F582E4346E
:1004960062F583E090610BF074032529F582E4345C
:1004A60062F583E090610CF074042529F582E4344A
:1004B60062F583E090610DF0E4A3F074052529F55B
:1004C60082E43463F583E090610FF074062529F524
:1004D60082E43463F583E0906110F074072529F512
:1004E60082E43463F583E0906111F074082529F500
:1004F60082E43463F583E0906112F07F11124E744A
:10050600220529E529C39440500302042FC208900E
:100516006618E0704130053E7478F0E4906102F0B0
:10052600A37408F0906405E0906104F0A374F0F001
:10053600E4A3F0A37490F0A37408F0E4A3F0A3F08E
:10054600A3F0A3F0A3F0A3F0A3F0A3F0A3F0A3F00D
:100556007F11124E7422E508C394045070E50825F5
:10056600E0FF7403A807088002C333D8FCF52955B9
:100576001365297053E529F45213E4906102F0A340
:100586007408F0906405E0906104F0A374F0F0A3A1
:100596007402F0A37491F0E5082420A3F0E5083373
:1005A600333354F875F002A42406F582E5F034647A
:1005B600F58363A20190610963A2017F101236E5FB
:1005C6007F17124E740508220508020653E508C374
:1005D60094085076E50824FC25E0FF7403A8070874
:1005E6008002C333D8FCF529551465297058E529CE
:1005F600F45214E4906102F0A37408F0906405E0EC
:10060600906104F0A374F0F0A37402F0A37491F067
:10061600E50854032440A3F0E50833333354F87552
:10062600F002A42406F582E5F03464F58363A201A2
:1006360090610963A2017F101236E57F17124E748E
:1006460005085308072205088003E4F50890683B6F
:10065600E0701F906102F0A37408F0906405E090CA
:100666006104F0A37490F0E4A3F0A3F07F06124EA9
:100676007422906616E0FF7003020A19F52AE4F068
:10068600201D1F7E1B7FE0124190E52A54802439ED
:10069600F582E43466AF82FEE52A547FFDE4FB1260
:1006A600434BE52A7003020A19E52A5480FF2439D0
:1006B600F582E43466AD82F52B8D2CE4F512F51146
:1006C6008F29E529C3952A5018052CE52CAE2B70E9
:1006D60002052B14F5828E83E0FF12512105298035
:1006E600E1E51145126026301D03020A197E1B7FC3
:1006F600E8124190E52A54802439F582E43466AF45
:1007060082FEE52A547FFDE4FB12434B22E490630C
:1007160003F0A3F0D20D906186F0E52A54802439C7
:10072600F582E43466AF82F52B8F2C7402252CF506
:100736002CE4352BF52B852C82F583E0FF906405A0
:10074600E0FEEF6E6026301D03020A197E1B7FF362
:10075600124190E52A54802439F582E43466AF824A
:10076600FEE52A547FFDE4FB12434B22052CE52CC3
:100776007002052BF582852B83E0FFB43006E490EA
:100786006184F022EF64017003020A19EFB41805C0
:10079600D209D21022EFB4190B906301E0F513A32E
:1007A600E0F51422852C82852B83E0FF54F064F05B
:1007B60060030208A1906617EFF0052CE52C700285
:1007C600052BF582852B83E0FF64807033052CE5CD
:1007D6002C7002052BF582852B83E06440600302B2
:1007E6000A19D212052CE52C7002052BF582852BF1
:1007F60083E064086003020A19D205906618F022A5
:10080600EFB40127052CE52C7002052BF582852B0C
:1008160083E0644F6003020A1990683CE0700302AB
:100826000A197408250EF50EE4F022852C82852B14
:1008360083E06003020A19052CE52C7002052BF5EE
:1008460082852B83E064426003020A19052CE52C9D
:100856007002052BF582852B83E0906F65F0052CE1
:10086600E52C7002052BF582852B83E0906F66F0F0
:10087600052CE52C7002052BF582852B83E0906F05
:1008860067F0052CE52C7002052BF582852B83E09D
:10089600906F68F0D22DC205D21222852C82852B4C
:1008A60083E0FF64116008EF641260030209F7E554
:1008B6002A547F640E60030209F7201D077E1B7F02
:1008C600FA124190302B0E301D03020A197E1C7F4E
:1008D6000F12419022852C82852B83E0540314F558
:1008E6002A052CE52C7002052BF582852B83E0F575
:1008F6002930E709E4906F64F0906F69F0E52930DC
:10090600E60BE4906F64F0906F697410F0E529309F
:10091600E50B906F647401F0E4906F69F0E529309F
:10092600E40C906F647401F0906F697410F0E5291F
:1009360030E30B906F647402F0E4906F69F0E52980
:1009460030E20C906F647402F0906F697410F0E5F9
:100956002930E10B906F647403F0E4906F69F0E561
:100966002930E00C906F647403F0906F697410F096
:100976007402252CF52CE4352BF52B852C82F5837A
:10098600E0F52930E700E52930E607906F69E024B5
:1009960002F0E52930E507906F69E02404F0E529C7
:1009A60030E407906F69E02406F0E52930E307900C
:1009B6006F69E02408F0E52930E207906F69E024CA
:1009C6000AF0E52930E107906F69E0240CF0E5298B
:1009D60030E007906F69E0240EF0906F69E0252AF9
:1009E600F0D22BE4906185F0906F63F0906FEBF09E
:1009F60022201D1F7E1C7F1D124190E52A54802453
:100A060039F582E43466AF82FEE52A547FFDE4FBC5
:030A160012434B3D
:010A190022BA
:10478A0002125DE493A3F8E493A34003F68001F2D6
:10479A0008DFF48029E493A3F85407240CC8C33330
:1047AA00C4540F4420C8834004F456800146F6DFFF
:1047BA00E4800B0102040810204080905162E47EDC
:1047CA00019360BCA3FF543F30E509541FFEE493F4
:1047DA00A360010ECF54C025E060A840B8E493A3BB
:1047EA00FAE493A3F8E493A3C8C582C8CAC583CAE6
:1047FA00F0A3C8C582C8CAC583CADFE9DEE780BE9E
:015168000046
:102A3800BB010689828A83E0225002E722BBFE029C
:092A4800E32289828A83E49322CF
:102A5100BB010CE58229F582E5833AF583E022503A
:102A610006E92582F8E622BBFE06E92582F8E22284
:0D2A7100E58229F582E5833AF583E493229E
:102A7E00BC000BBE0029EF8DF084FFADF022E4CC3C
:102A8E00F875F008EF2FFFEE33FEEC33FCEE9DEC05
:102A9E00984005FCEE9DFE0FD5F0E9E4CEFD22ED4B
:102AAE00F8F5F0EE8420D21CFEADF075F008EF2F95
:102ABE00FFED33FD4007985006D5F0F222C398FD86
:052ACE000FD5F0EA2223
:102AD30075F008758200EF2FFFEE33FECD33CDCCBA
:102AE30033CCC58233C5829BED9AEC99E58298403D
:102AF3000CF582EE9BFEED9AFDEC99FC0FD5F0D61A
:102B0300E4CEFBE4CDFAE4CCF9A88222B800C1B943
:102B13000059BA002DEC8BF084CFCECDFCE5F0CB81
:102B2300F97818EF2FFFEE33FEED33FDEC33FCEBBA
:102B330033FB10D703994004EB99FB0FD8E5E4F975
:102B4300FA227818EF2FFFEE33FEED33FDEC33FC62
:102B5300C933C910D7059BE99A4007EC9BFCE99A56
:102B6300F90FD8E0E4C9FAE4CCFB2275F010EF2F9B
:102B7300FFEE33FEED33FDCC33CCC833C810D7079B
:102B83009BEC9AE899400AED9BFDEC9AFCE899F8D6
:0E2B93000FD5F0DAE4CDFBE4CCFAE4C8F92269
:0E2BA100C3E49FFFE49EFEE49DFDE49CFC2245
:102BAF00EB9FF5F0EA9E42F0E99D42F0E89C45F07C
:012BBF0022F3
:0C2BC000ECF0A3EDF0A3EEF0A3EFF02288
:102BCC00A8828583F0D083D082122BE3122BE312E0
:102BDC002BE3122BE3E473E493A3C583C5F0C58305
:102BEC00C8C582C8F0A3C583C5F0C583C8C582C853
:012BFC0022B6
:1023C000E53C2430F8E6053C22782D3029027830AF
:1023D000E475F001122C5E022A382022EB7F2ED207
:1023E000228018EF540F2490D43440D4FF30260BB1
:1023F000EF24BFB41A0050032461FFE53D600215CD
:102400003D0540E5407002053F30290D782DE4750B
:10241000F001122C5EEF022BFD024E2D7403D22927
:102420008003E4C229F53C8B2D8A2E892FE4F53DEB
:10243000F53FF540E53D60077F201223FB80F575F1
:102440003EFFC223C222C224C225C227C228C22AFA
:102450001223C9FF700D3029057F0012240CAF40F4
:10246000AE3F22B4255FC2D5C2261223C9FF24D0B5
:10247000B40A00501A75F00A783D30D50508B6FF49
:102480000106C6A426F620D5047002D22580D924E0
:10249000CFB41A00EF5004C2E5D22602260CD22394
:1024A00080C6D22280C0D22480BCD2D580BAD227A6
:1024B00080B47F201223FB2024077401B53D004027
:1024C000F11223C0FF1223FB022434D22AD2288027
:1024D000951223C0FB1223C0FA1223C0F94A4B7095
:1024E0000679DD7A267BFF20242EE53D602A7E00DA
:1024F0008E82758300122A5160060EEE653E70F0E2
:10250000C2D5EBC0E0EAC0E0E9C0E0EE122653D04D
:10251000E0F9D0E0FAD0E0FB122A38FF60AAEBC065
:10252000E0EAC0E0E9C0E01223FBD0E02401F9D0EA
:10253000E03400FAD0E0FBE53E0460DCD53ED98013
:10254000877BFF7A26794FD224809C79108002798C
:1025500008C228C22A8008D2D5790A8004790AC222
:10256000D5E53E047002F53EE4FAFDFEFF1223C0FD
:10257000FC7B082023131223C0FD7B1030220A129B
:1025800023C0FE1223C0FF7B20EC3382D592D550AE
:1025900013C3E43022069FFFE49EFEE42023039D44
:1025A000FDE49CFCE4CBF8C223EC700CCFCECDCC88
:1025B000E824F8F870F38017C3EF33FFEE33FEED35
:1025C00033FDEC33FCEB33FB994002FB0FD8E9EB16
:1025D000302305F8D0E0C448B223C0E00AEC4D4EE9
:1025E0004F78207B0070C2EAB53E0040BCC0E012CC
:1025F0002655D0F0D0E0202304C4C0E0C4B223C0EC
:10260000F01223E4D0F0D5F0EB022434122CBD24D8
:10261000D153254B5824A24C249E42254F4F255779
:0F2620004425574924B743255D5525414625419B
:10262F004525414726FD5024A62D24AA2E24CD2B27
:10263F0024AE2324CB2026E62A246648000024C596
:10264F003F3F3F00790AA2D5202514302709B91042
:10265F00020404B9080104A2D52028025001042065
:10266F0024689224B53D005034C0E07F20302519F6
:10267F007F30A22472287227500F1226ACC224C2B8
:10268F0028C227C22A7F30800F302703E9C0E0120B
:10269F0023FB302703D0E0F9D0E0B53DCC3027172E
:1026AF007F30B9100C1223FB7F583026077F7880BC
:1026BF0003B908031223FB3024057F2D0223FB7F70
:1026CF0020202AF87F2B2028F322922480CF286EF7
:1026DF00756C6C2900D2231223C03023F8C22378E3
:1026EF003D30D50108F60224662D50434958122378
:1026FF00C02403B405004001E49026F8931223ECA4
:0D270F00743A1223ECD225753D0402254BCF
:1037BC008B308A318932E4F53CF53BF53AF539F535
:1037CC0037F538E534453545336012EBC0E0EAC0D7
:1037DC00E0E9C0E0AB33AA34A935122C6EAB30054E
:1037EC0032E532AA317002053114F9122A38F53D4E
:1037FC00C394094007E53DD3940D40E1E53D6420B9
:10380C0060DBE53DB42D054338038016E53DB42B54
:10381C0005433801800C74FF2532F53274FF3531C5
:10382C00F531E53660046410703FAB30AA31A93233
:10383C00122A3864306009E536702E75360A8029F4
:10384C00900001122A51FF64786004EFB4581343BE
:10385C00380175361074022532F532E43531F53104
:10386C008007E5367003753608AB300532E532AAB1
:10387C00317002053114F9122A38F53DC3946140B8
:10388C000AE53DD3947A5003533DDF74D0253DF5C2
:10389C003DC3940A400CE53D9411406D74F9253DEF
:1038AC00F53DE53DD395365060433801853C418567
:1038BC003B40853A3F85393EAF367E00E4FCFDAB9C
:1038CC003CAA3BA93AA839122C0FC8ECC8C9EDC9BF
:1038DC00CAEECACBEFCBE4FCFDFEEB253DF53CEE8E
:1038EC003AF53BED39F53AEC38F539AF3CAE3BAD3A
:1038FC003AFCAB41AA40A93FA83ED3122BAF5003D0
:10390C00023875433804023875E53820E003E4804A
:10391C002DE53445354533601EAB30E53224FFF9D7
:10392C00E53134FFFAEBC0E0EAC0E0E9C0E0AB33CC
:10393C00AA34A935122C6EE53830E20774FFFFFE6D
:10394C00FDFC22E538AF3CAE3BAD3AAC3930E1037F
:04395C00022BA12277
:102BFD00BB010689828A83F0225002F722BBFE01B7
:022C0D00F322B0
:102C0F00E88FF0A4CC8BF0A42CFCE98EF0A42CFC64
:102C1F008AF0EDA42CFCEA8EF0A4CDA8F08BF0A4E2
:102C2F002DCC3825F0FDE98FF0A42CCD35F0FCEB41
:102C3F008EF0A4FEA9F0EB8FF0A4CFC5F02ECD3906
:0F2C4F00FEE43CFCEAA42DCE35F0FDE43CFC2273
:102C5E00FAE6FB0808E6F925F0F618E6CA3AF62277
:102C6E00BB011A89828A83D0F0D0E0F8D0E0F9D087
:102C7E00E0FAD0E0FBE8C0E0C0F0022CEC5016E920
:102C8E00F8D083D082D0E0F9D0E0FAD0E0FBC08259
:102C9E00C083022CE3BBFE16E9F8D083D082D0E0CD
:0F2CAE00F9D0E0FAD0E0FBC082C083022CF522FF
:102CBD00D083D082F8E4937012740193700DA3A3A6
:102CCD0093F8740193F5828883E4737402936860BA
:062CDD00EFA3A3A380DFBA
:092CE300EBF608EAF608E9F62216
:092CEC00EBF0A3EAF0A3E9F022E9
:092CF500EBF208EAF208E9F22210
:00000001FF
